Archive member included to satisfy reference by file (symbol)

.\CortexM3\ARM_GCC_541\Debug\Serrure.a(CyLib.o)
                              .\CortexM3\ARM_GCC_541\Debug\Cm3Start.o (CyHalt)
.\CortexM3\ARM_GCC_541\Debug\Serrure.a(cyPm.o)
                              .\CortexM3\ARM_GCC_541\Debug\Serrure.a(CyLib.o) (CyPmReadStatus)
.\CortexM3\ARM_GCC_541\Debug\Serrure.a(UART.o)
                              .\CortexM3\ARM_GCC_541\Debug\main.o (UART_Start)
.\CortexM3\ARM_GCC_541\Debug\Serrure.a(UART_INT.o)
                              .\CortexM3\ARM_GCC_541\Debug\Serrure.a(UART.o) (UART_RXISR)
.\CortexM3\ARM_GCC_541\Debug\Serrure.a(UART_IntClock.o)
                              .\CortexM3\ARM_GCC_541\Debug\Serrure.a(UART.o) (UART_IntClock_Start)
.\CortexM3\ARM_GCC_541\Debug\Serrure.a(rfid.o)
                              .\CortexM3\ARM_GCC_541\Debug\main.o (rfid_Start)
.\CortexM3\ARM_GCC_541\Debug\Serrure.a(led.o)
                              .\CortexM3\ARM_GCC_541\Debug\Serrure.a(rfid.o) (led_Write)
.\CortexM3\ARM_GCC_541\Debug\Serrure.a(CyBootAsmGnu.o)
                              .\CortexM3\ARM_GCC_541\Debug\cyfitter_cfg.o (CyDelayCycles)
.\CortexM3\ARM_GCC_541\Debug\Serrure.a(CyFlash.o)
                              .\CortexM3\ARM_GCC_541\Debug\Serrure.a(cyPm.o) (CyFlash_SetWaitCycles)
.\CortexM3\ARM_GCC_541\Debug\Serrure.a(CySpc.o)
                              .\CortexM3\ARM_GCC_541\Debug\Serrure.a(CyFlash.o) (CySpcStart)
c:/program files (x86)/cypress/psoc creator/4.2/psoc creator/import/gnu/arm/5.4.1/bin/../lib/gcc/arm-none-eabi/5.4.1/../../../../arm-none-eabi/lib/armv7-m\libg_nano.a(lib_a-errno.o)
                              .\CortexM3\ARM_GCC_541\Debug\Cm3Start.o (__errno)
c:/program files (x86)/cypress/psoc creator/4.2/psoc creator/import/gnu/arm/5.4.1/bin/../lib/gcc/arm-none-eabi/5.4.1/../../../../arm-none-eabi/lib/armv7-m\libg_nano.a(lib_a-exit.o)
                              c:/program files (x86)/cypress/psoc creator/4.2/psoc creator/import/gnu/arm/5.4.1/bin/../lib/gcc/arm-none-eabi/5.4.1/../../../../arm-none-eabi/lib/armv7-m/crt0.o (exit)
c:/program files (x86)/cypress/psoc creator/4.2/psoc creator/import/gnu/arm/5.4.1/bin/../lib/gcc/arm-none-eabi/5.4.1/../../../../arm-none-eabi/lib/armv7-m\libg_nano.a(lib_a-impure.o)
                              c:/program files (x86)/cypress/psoc creator/4.2/psoc creator/import/gnu/arm/5.4.1/bin/../lib/gcc/arm-none-eabi/5.4.1/../../../../arm-none-eabi/lib/armv7-m\libg_nano.a(lib_a-exit.o) (_global_impure_ptr)
c:/program files (x86)/cypress/psoc creator/4.2/psoc creator/import/gnu/arm/5.4.1/bin/../lib/gcc/arm-none-eabi/5.4.1/../../../../arm-none-eabi/lib/armv7-m\libg_nano.a(lib_a-init.o)
                              c:/program files (x86)/cypress/psoc creator/4.2/psoc creator/import/gnu/arm/5.4.1/bin/../lib/gcc/arm-none-eabi/5.4.1/../../../../arm-none-eabi/lib/armv7-m/crt0.o (__libc_init_array)
c:/program files (x86)/cypress/psoc creator/4.2/psoc creator/import/gnu/arm/5.4.1/bin/../lib/gcc/arm-none-eabi/5.4.1/../../../../arm-none-eabi/lib/armv7-m\libg_nano.a(lib_a-memcpy-stub.o)
                              .\CortexM3\ARM_GCC_541\Debug\cyfitter_cfg.o (memcpy)
c:/program files (x86)/cypress/psoc creator/4.2/psoc creator/import/gnu/arm/5.4.1/bin/../lib/gcc/arm-none-eabi/5.4.1/../../../../arm-none-eabi/lib/armv7-m\libg_nano.a(lib_a-memset.o)
                              c:/program files (x86)/cypress/psoc creator/4.2/psoc creator/import/gnu/arm/5.4.1/bin/../lib/gcc/arm-none-eabi/5.4.1/../../../../arm-none-eabi/lib/armv7-m/crt0.o (memset)

Allocating common symbols
Common symbol       size              file

UART_rxBuffer       0x5               .\CortexM3\ARM_GCC_541\Debug\Serrure.a(UART.o)
dieTemperature      0x2               .\CortexM3\ARM_GCC_541\Debug\Serrure.a(CyFlash.o)

Discarded input sections

 .text          0x00000000        0x0 c:/program files (x86)/cypress/psoc creator/4.2/psoc creator/import/gnu/arm/5.4.1/bin/../lib/gcc/arm-none-eabi/5.4.1/armv7-m/crti.o
 .data          0x00000000        0x0 c:/program files (x86)/cypress/psoc creator/4.2/psoc creator/import/gnu/arm/5.4.1/bin/../lib/gcc/arm-none-eabi/5.4.1/armv7-m/crti.o
 .bss           0x00000000        0x0 c:/program files (x86)/cypress/psoc creator/4.2/psoc creator/import/gnu/arm/5.4.1/bin/../lib/gcc/arm-none-eabi/5.4.1/armv7-m/crti.o
 .data          0x00000000        0x4 c:/program files (x86)/cypress/psoc creator/4.2/psoc creator/import/gnu/arm/5.4.1/bin/../lib/gcc/arm-none-eabi/5.4.1/armv7-m/crtbegin.o
 .text          0x00000000       0x74 c:/program files (x86)/cypress/psoc creator/4.2/psoc creator/import/gnu/arm/5.4.1/bin/../lib/gcc/arm-none-eabi/5.4.1/../../../../arm-none-eabi/lib/armv7-m/crt0.o
 .data          0x00000000        0x0 c:/program files (x86)/cypress/psoc creator/4.2/psoc creator/import/gnu/arm/5.4.1/bin/../lib/gcc/arm-none-eabi/5.4.1/../../../../arm-none-eabi/lib/armv7-m/crt0.o
 .bss           0x00000000        0x0 c:/program files (x86)/cypress/psoc creator/4.2/psoc creator/import/gnu/arm/5.4.1/bin/../lib/gcc/arm-none-eabi/5.4.1/../../../../arm-none-eabi/lib/armv7-m/crt0.o
 .ARM.extab     0x00000000        0x0 c:/program files (x86)/cypress/psoc creator/4.2/psoc creator/import/gnu/arm/5.4.1/bin/../lib/gcc/arm-none-eabi/5.4.1/../../../../arm-none-eabi/lib/armv7-m/crt0.o
 .ARM.exidx     0x00000000        0x8 c:/program files (x86)/cypress/psoc creator/4.2/psoc creator/import/gnu/arm/5.4.1/bin/../lib/gcc/arm-none-eabi/5.4.1/../../../../arm-none-eabi/lib/armv7-m/crt0.o
 .text          0x00000000        0x0 .\CortexM3\ARM_GCC_541\Debug\main.o
 .data          0x00000000        0x0 .\CortexM3\ARM_GCC_541\Debug\main.o
 .bss           0x00000000        0x0 .\CortexM3\ARM_GCC_541\Debug\main.o
 .text          0x00000000        0x0 .\CortexM3\ARM_GCC_541\Debug\cyfitter_cfg.o
 .data          0x00000000        0x0 .\CortexM3\ARM_GCC_541\Debug\cyfitter_cfg.o
 .bss           0x00000000        0x0 .\CortexM3\ARM_GCC_541\Debug\cyfitter_cfg.o
 .text.SetAnalogRoutingPumps
                0x00000000       0x10 .\CortexM3\ARM_GCC_541\Debug\cyfitter_cfg.o
 .text          0x00000000        0x0 .\CortexM3\ARM_GCC_541\Debug\cymetadata.o
Memory Configuration

Name             Origin             Length             Attributes
rom              0x00000000         0x00040000         xr
ram              0x1fff8000         0x00010000         xrw
*default*        0x00000000         0xffffffff

Linker script and memory map

LOAD c:/program files (x86)/cypress/psoc creator/4.2/psoc creator/import/gnu/arm/5.4.1/bin/../lib/gcc/arm-none-eabi/5.4.1/armv7-m/crti.o
LOAD c:/program files (x86)/cypress/psoc creator/4.2/psoc creator/import/gnu/arm/5.4.1/bin/../lib/gcc/arm-none-eabi/5.4.1/armv7-m/crtbegin.o
LOAD c:/program files (x86)/cypress/psoc creator/4.2/psoc creator/import/gnu/arm/5.4.1/bin/../lib/gcc/arm-none-eabi/5.4.1/../../../../arm-none-eabi/lib/armv7-m/crt0.o
START GROUP
LOAD .\CortexM3\ARM_GCC_541\Debug\main.o
LOAD .\CortexM3\ARM_GCC_541\Debug\cyfitter_cfg.o
LOAD .\CortexM3\ARM_GCC_541\Debug\cymetadata.o
LOAD .\CortexM3\ARM_GCC_541\Debug\Cm3Start.o
LOAD .\CortexM3\ARM_GCC_541\Debug\Serrure.a
LOAD C:\Program Files (x86)\Cypress\PSoC Creator\4.2\PSoC Creator\psoc\content\cycomponentlibrary\CyComponentLibrary.cylib\CortexM3\ARM_GCC_541\Debug\CyComponentLibrary.a
END GROUP
START GROUP
LOAD c:/program files (x86)/cypress/psoc creator/4.2/psoc creator/import/gnu/arm/5.4.1/bin/../lib/gcc/arm-none-eabi/5.4.1/armv7-m\libgcc.a
LOAD c:/program files (x86)/cypress/psoc creator/4.2/psoc creator/import/gnu/arm/5.4.1/bin/../lib/gcc/arm-none-eabi/5.4.1/../../../../arm-none-eabi/lib/armv7-m\libg_nano.a
LOAD c:/program files (x86)/cypress/psoc creator/4.2/psoc creator/import/gnu/arm/5.4.1/bin/../lib/gcc/arm-none-eabi/5.4.1/../../../../arm-none-eabi/lib/armv7-m\libc_nano.a
END GROUP
START GROUP
LOAD c:/program files (x86)/cypress/psoc creator/4.2/psoc creator/import/gnu/arm/5.4.1/bin/../lib/gcc/arm-none-eabi/5.4.1/armv7-m\libgcc.a
LOAD c:/program files (x86)/cypress/psoc creator/4.2/psoc creator/import/gnu/arm/5.4.1/bin/../lib/gcc/arm-none-eabi/5.4.1/../../../../arm-none-eabi/lib/armv7-m\libc_nano.a
END GROUP
LOAD c:/program files (x86)/cypress/psoc creator/4.2/psoc creator/import/gnu/arm/5.4.1/bin/../lib/gcc/arm-none-eabi/5.4.1/armv7-m/crtend.o
LOAD c:/program files (x86)/cypress/psoc creator/4.2/psoc creator/import/gnu/arm/5.4.1/bin/../lib/gcc/arm-none-eabi/5.4.1/armv7-m/crtn.o
START GROUP
LOAD c:/program files (x86)/cypress/psoc creator/4.2/psoc creator/import/gnu/arm/5.4.1/bin/../lib/gcc/arm-none-eabi/5.4.1/armv7-m\libgcc.a
LOAD c:/program files (x86)/cypress/psoc creator/4.2/psoc creator/import/gnu/arm/5.4.1/bin/../lib/gcc/arm-none-eabi/5.4.1/../../../../arm-none-eabi/lib/armv7-m\libc.a
LOAD c:/program files (x86)/cypress/psoc creator/4.2/psoc creator/import/gnu/arm/5.4.1/bin/../lib/gcc/arm-none-eabi/5.4.1/../../../../arm-none-eabi/lib/armv7-m\libnosys.a
END GROUP
                0x00000000                CY_APPL_ORIGIN = 0x0
                0x00000100                CY_FLASH_ROW_SIZE = 0x100
                0x00000020                CY_ECC_ROW_SIZE = 0x20
                0x00000000                CY_EE_IN_BTLDR = 0x0
                0x00000000                CY_APPL_LOADABLE = 0x0
                0x00000800                CY_EE_SIZE = 0x800
                0x00000001                CY_APPL_NUM = 0x1
                0x00000001                CY_APPL_MAX = 0x1
                0x00000040                CY_METADATA_SIZE = 0x40
                0x00000000                CY_APPL_LOADABLE = 0x0
                0x00000000                CY_CHECKSUM_EXCLUDE_SIZE = ALIGN (0x0, CY_FLASH_ROW_SIZE)
                [!provide]                PROVIDE (__cy_heap_start, _end)
                0x00000001                PROVIDE (__cy_region_num, ((__cy_regions_end - __cy_regions) / 0x10))
                0x20008000                PROVIDE (__cy_stack, (ORIGIN (ram) + LENGTH (ram)))
                [!provide]                PROVIDE (__cy_heap_end, (__cy_stack - 0x800))

.cybootloader   0x00000000        0x0
 *(.cybootloader)
                0x00000000                appl1_start = CY_APPL_ORIGIN?CY_APPL_ORIGIN:ALIGN (CY_FLASH_ROW_SIZE)
                0x0001ff00                appl2_start = (appl1_start + ALIGN ((((LENGTH (rom) - appl1_start) - (0x2 * CY_FLASH_ROW_SIZE)) / 0x2), CY_FLASH_ROW_SIZE))
                0x00000000                appl_start = (CY_APPL_NUM == 0x1)?appl1_start:appl2_start
                0x00000000                ecc_offset = ((appl_start / CY_FLASH_ROW_SIZE) * CY_ECC_ROW_SIZE)
                0x00000000                ee_offset = (CY_APPL_LOADABLE && ! (CY_EE_IN_BTLDR))?((CY_EE_SIZE / CY_APPL_MAX) * (CY_APPL_NUM - 0x1)):0x0
                0x00000800                ee_size = (CY_APPL_LOADABLE && ! (CY_EE_IN_BTLDR))?(CY_EE_SIZE / CY_APPL_MAX):CY_EE_SIZE
                [!provide]                PROVIDE (CY_ECC_OFFSET, ecc_offset)

.text           0x00000000      0x84e
 CREATE_OBJECT_SYMBOLS
                0x00000000                PROVIDE (__cy_interrupt_vector, RomVectors)
 *(.romvectors)
 .romvectors    0x00000000       0x10 .\CortexM3\ARM_GCC_541\Debug\Cm3Start.o
                0x00000000                RomVectors
                0x00000001                ASSERT ((. != __cy_interrupt_vector), No interrupt vector)
                0x00000001                ASSERT (CY_APPL_ORIGIN?(SIZEOF (.cybootloader) <= CY_APPL_ORIGIN):0x1, Wrong image location)
                0x00000010                PROVIDE (__cy_reset, Reset)
 *(.text.Reset)
 .text.Reset    0x00000010       0x18 .\CortexM3\ARM_GCC_541\Debug\Cm3Start.o
                0x00000010                Reset
                0x00000001                ASSERT ((. != __cy_reset), No reset code)
 *(.dma_init)
                0x00000001                ASSERT ((((appl_start + .) <= 0x10000) || 0x1), DMA Init must be within the first 64k of flash)
 *(.text .text.* .gnu.linkonce.t.*)
 .text          0x00000028       0x5c c:/program files (x86)/cypress/psoc creator/4.2/psoc creator/import/gnu/arm/5.4.1/bin/../lib/gcc/arm-none-eabi/5.4.1/armv7-m/crtbegin.o
 .text.main     0x00000084       0x18 .\CortexM3\ARM_GCC_541\Debug\main.o
                0x00000084                main
 .text.CyClockStartupError
                0x0000009c        0x4 .\CortexM3\ARM_GCC_541\Debug\cyfitter_cfg.o
 .text.cfg_write_bytes32
                0x000000a0       0x34 .\CortexM3\ARM_GCC_541\Debug\cyfitter_cfg.o
 .text.AnalogSetDefault
                0x000000d4       0x28 .\CortexM3\ARM_GCC_541\Debug\cyfitter_cfg.o
 .text.CYMEMZERO
                0x000000fc        0xc .\CortexM3\ARM_GCC_541\Debug\cyfitter_cfg.o
 .text.ClockSetup
                0x00000108       0xcc .\CortexM3\ARM_GCC_541\Debug\cyfitter_cfg.o
 .text.CYCONFIGCPY
                0x000001d4        0x8 .\CortexM3\ARM_GCC_541\Debug\cyfitter_cfg.o
 .text.cyfitter_cfg
                0x000001dc      0x110 .\CortexM3\ARM_GCC_541\Debug\cyfitter_cfg.o
                0x000001dc                cyfitter_cfg
 .text.IntDefaultHandler
                0x000002ec       0x10 .\CortexM3\ARM_GCC_541\Debug\Cm3Start.o
                0x000002ec                IntDefaultHandler
 .text.Start_c  0x000002fc       0x4c .\CortexM3\ARM_GCC_541\Debug\Cm3Start.o
                0x000002fc                Start_c
 .text.initialize_psoc
                0x00000348       0x68 .\CortexM3\ARM_GCC_541\Debug\Cm3Start.o
                0x00000348                initialize_psoc
 .text.CyHalt   0x000003b0        0x4 .\CortexM3\ARM_GCC_541\Debug\Serrure.a(CyLib.o)
                0x000003b0                CyHalt
 .text.CyDelay  0x000003b4       0x2c .\CortexM3\ARM_GCC_541\Debug\Serrure.a(CyLib.o)
                0x000003b4                CyDelay
 .text.CyIntSetVector
                0x000003e0       0x28 .\CortexM3\ARM_GCC_541\Debug\Serrure.a(CyLib.o)
                0x000003e0                CyIntSetVector
 .text.CyIntSetPriority
                0x00000408       0x30 .\CortexM3\ARM_GCC_541\Debug\Serrure.a(CyLib.o)
                0x00000408                CyIntSetPriority
 .text.UART_Init
                0x00000438       0x44 .\CortexM3\ARM_GCC_541\Debug\Serrure.a(UART.o)
                0x00000438                UART_Init
 .text.UART_Enable
                0x0000047c       0x48 .\CortexM3\ARM_GCC_541\Debug\Serrure.a(UART.o)
                0x0000047c                UART_Enable
 .text.UART_Start
                0x000004c4       0x1c .\CortexM3\ARM_GCC_541\Debug\Serrure.a(UART.o)
                0x000004c4                UART_Start
 .text.UART_GetChar
                0x000004e0       0x80 .\CortexM3\ARM_GCC_541\Debug\Serrure.a(UART.o)
                0x000004e0                UART_GetChar
 .text.UART_GetRxBufferSize
                0x00000560       0x60 .\CortexM3\ARM_GCC_541\Debug\Serrure.a(UART.o)
                0x00000560                UART_GetRxBufferSize
 .text.UART_PutChar
                0x000005c0       0x18 .\CortexM3\ARM_GCC_541\Debug\Serrure.a(UART.o)
                0x000005c0                UART_PutChar
 .text.UART_PutString
                0x000005d8       0x24 .\CortexM3\ARM_GCC_541\Debug\Serrure.a(UART.o)
                0x000005d8                UART_PutString
 .text.UART_PutArray
                0x000005fc       0x28 .\CortexM3\ARM_GCC_541\Debug\Serrure.a(UART.o)
                0x000005fc                UART_PutArray
 .text.UART_RXISR
                0x00000624       0x98 .\CortexM3\ARM_GCC_541\Debug\Serrure.a(UART_INT.o)
                0x00000624                UART_RXISR
 .text.UART_IntClock_Start
                0x000006bc       0x1c .\CortexM3\ARM_GCC_541\Debug\Serrure.a(UART_IntClock.o)
                0x000006bc                UART_IntClock_Start
 .text.rfid_Interrupt
                0x000006d8       0x6c .\CortexM3\ARM_GCC_541\Debug\Serrure.a(rfid.o)
                0x000006d8                rfid_Interrupt
 .text.rfid_SetVector
                0x00000744        0xc .\CortexM3\ARM_GCC_541\Debug\Serrure.a(rfid.o)
                0x00000744                rfid_SetVector
 .text.rfid_SetPriority
                0x00000750       0x10 .\CortexM3\ARM_GCC_541\Debug\Serrure.a(rfid.o)
                0x00000750                rfid_SetPriority
 .text.rfid_Enable
                0x00000760        0xc .\CortexM3\ARM_GCC_541\Debug\Serrure.a(rfid.o)
                0x00000760                rfid_Enable
 .text.rfid_Disable
                0x0000076c        0xc .\CortexM3\ARM_GCC_541\Debug\Serrure.a(rfid.o)
                0x0000076c                rfid_Disable
 .text.rfid_Start
                0x00000778       0x1c .\CortexM3\ARM_GCC_541\Debug\Serrure.a(rfid.o)
                0x00000778                rfid_Start
 .text.led_Write
                0x00000794       0x18 .\CortexM3\ARM_GCC_541\Debug\Serrure.a(led.o)
                0x00000794                led_Write
 *fill*         0x000007ac        0x4 
 .text          0x000007b0       0x20 .\CortexM3\ARM_GCC_541\Debug\Serrure.a(CyBootAsmGnu.o)
                0x000007b0                CyDelayCycles
                0x000007c0                CyEnterCriticalSection
                0x000007c8                CyExitCriticalSection
 .text.__errno  0x000007d0        0xc c:/program files (x86)/cypress/psoc creator/4.2/psoc creator/import/gnu/arm/5.4.1/bin/../lib/gcc/arm-none-eabi/5.4.1/../../../../arm-none-eabi/lib/armv7-m\libg_nano.a(lib_a-errno.o)
                0x000007d0                __errno
 .text.__libc_init_array
                0x000007dc       0x4c c:/program files (x86)/cypress/psoc creator/4.2/psoc creator/import/gnu/arm/5.4.1/bin/../lib/gcc/arm-none-eabi/5.4.1/../../../../arm-none-eabi/lib/armv7-m\libg_nano.a(lib_a-init.o)
                0x000007dc                __libc_init_array
 .text.memcpy   0x00000828       0x16 c:/program files (x86)/cypress/psoc creator/4.2/psoc creator/import/gnu/arm/5.4.1/bin/../lib/gcc/arm-none-eabi/5.4.1/../../../../arm-none-eabi/lib/armv7-m\libg_nano.a(lib_a-memcpy-stub.o)
                0x00000828                memcpy
 .text.memset   0x0000083e       0x10 c:/program files (x86)/cypress/psoc creator/4.2/psoc creator/import/gnu/arm/5.4.1/bin/../lib/gcc/arm-none-eabi/5.4.1/../../../../arm-none-eabi/lib/armv7-m\libg_nano.a(lib_a-memset.o)
                0x0000083e                memset
 *(.plt)
 *(.gnu.warning)
 *(.glue_7t)
 .glue_7t       0x0000084e        0x0 linker stubs
 *(.glue_7)
 .glue_7        0x0000084e        0x0 linker stubs
 *(.vfp11_veneer)
 .vfp11_veneer  0x0000084e        0x0 linker stubs
 *(.bootloader)
 *(.ARM.extab* .gnu.linkonce.armextab.*)
 *(.gcc_except_table)

.v4_bx          0x00000850        0x0
 .v4_bx         0x00000850        0x0 linker stubs

.iplt           0x00000850        0x0
 .iplt          0x00000850        0x0 c:/program files (x86)/cypress/psoc creator/4.2/psoc creator/import/gnu/arm/5.4.1/bin/../lib/gcc/arm-none-eabi/5.4.1/armv7-m/crtbegin.o

.eh_frame_hdr
 *(.eh_frame_hdr)

.eh_frame       0x00000850        0x4
 *(.eh_frame)
 .eh_frame      0x00000850        0x0 c:/program files (x86)/cypress/psoc creator/4.2/psoc creator/import/gnu/arm/5.4.1/bin/../lib/gcc/arm-none-eabi/5.4.1/armv7-m/crtbegin.o
 .eh_frame      0x00000850        0x4 c:/program files (x86)/cypress/psoc creator/4.2/psoc creator/import/gnu/arm/5.4.1/bin/../lib/gcc/arm-none-eabi/5.4.1/armv7-m/crtend.o
                [!provide]                PROVIDE (__exidx_start, .)

.ARM.exidx
 *(.ARM.exidx* .gnu.linkonce.armexidx.*)
                0x00000854                __exidx_end = .

.rodata         0x00000854       0x9c
 *(.rodata .rodata.* .gnu.linkonce.r.*)
 .rodata.str1.4
                0x00000854        0x9 .\CortexM3\ARM_GCC_541\Debug\main.o
 *fill*         0x0000085d        0x3 
 .rodata        0x00000860       0x46 .\CortexM3\ARM_GCC_541\Debug\cyfitter_cfg.o
 *fill*         0x000008a6        0x2 
 .rodata.str1.4
                0x000008a8        0xc .\CortexM3\ARM_GCC_541\Debug\Serrure.a(rfid.o)
                                  0xf (size before relaxing)
 .rodata.str1.1
                0x000008b4        0x2 c:/program files (x86)/cypress/psoc creator/4.2/psoc creator/import/gnu/arm/5.4.1/bin/../lib/gcc/arm-none-eabi/5.4.1/../../../../arm-none-eabi/lib/armv7-m\libg_nano.a(lib_a-impure.o)
                0x000008b8                . = ALIGN (0x4)
 *fill*         0x000008b6        0x2 
 *(.init)
 .init          0x000008b8        0x4 c:/program files (x86)/cypress/psoc creator/4.2/psoc creator/import/gnu/arm/5.4.1/bin/../lib/gcc/arm-none-eabi/5.4.1/armv7-m/crti.o
                0x000008b8                _init
 .init          0x000008bc        0x8 c:/program files (x86)/cypress/psoc creator/4.2/psoc creator/import/gnu/arm/5.4.1/bin/../lib/gcc/arm-none-eabi/5.4.1/armv7-m/crtn.o
                0x000008c4                . = ALIGN (0x4)
                0x000008c4                __preinit_array_start = .
 *(.preinit_array)
                0x000008c4                __preinit_array_end = .
                0x000008c4                . = ALIGN (0x4)
                0x000008c4                __init_array_start = .
 *(SORT(.init_array.*))
 *(.init_array)
 .init_array    0x000008c4        0x4 c:/program files (x86)/cypress/psoc creator/4.2/psoc creator/import/gnu/arm/5.4.1/bin/../lib/gcc/arm-none-eabi/5.4.1/armv7-m/crtbegin.o
 .init_array    0x000008c8        0x4 .\CortexM3\ARM_GCC_541\Debug\Cm3Start.o
                0x000008cc                __init_array_end = .
                0x000008cc                . = ALIGN (0x4)
 *(.fini)
 .fini          0x000008cc        0x4 c:/program files (x86)/cypress/psoc creator/4.2/psoc creator/import/gnu/arm/5.4.1/bin/../lib/gcc/arm-none-eabi/5.4.1/armv7-m/crti.o
                0x000008cc                _fini
 .fini          0x000008d0        0x8 c:/program files (x86)/cypress/psoc creator/4.2/psoc creator/import/gnu/arm/5.4.1/bin/../lib/gcc/arm-none-eabi/5.4.1/armv7-m/crtn.o
                0x000008d8                . = ALIGN (0x4)
                0x000008d8                __fini_array_start = .
 *(.fini_array)
 .fini_array    0x000008d8        0x4 c:/program files (x86)/cypress/psoc creator/4.2/psoc creator/import/gnu/arm/5.4.1/bin/../lib/gcc/arm-none-eabi/5.4.1/armv7-m/crtbegin.o
 *(SORT(.fini_array.*))
                0x000008dc                __fini_array_end = .
                0x000008dc                . = ALIGN (0x4)
 *crtbegin.o(.ctors)
 *(EXCLUDE_FILE(*crtend.o) .ctors)
 *(SORT(.ctors.*))
 *crtend.o(.ctors)
                0x000008dc                . = ALIGN (0x4)
 *crtbegin.o(.dtors)
 *(EXCLUDE_FILE(*crtend.o) .dtors)
 *(SORT(.dtors.*))
 *crtend.o(.dtors)
                0x000008dc                . = ALIGN (0x4)
                0x000008dc                __cy_regions = .
                0x000008dc        0x4 LONG 0x8f0 __cy_region_init_ram
                0x000008e0        0x4 LONG 0x1fff80c8 __cy_region_start_data
                0x000008e4        0x4 LONG 0x78 __cy_region_init_size_ram
                0x000008e8        0x4 LONG 0x30 __cy_region_zero_size_ram
                0x000008ec                __cy_regions_end = .
                0x000008f0                . = ALIGN (0x8)
 *fill*         0x000008ec        0x4 
                0x000008f0                _etext = .

.cy_checksum_exclude
                0x000008f0        0x0
 *(.cy_checksum_exclude)

.ramvectors     0x1fff8000       0xc0
                0x1fff8000                __cy_region_start_ram = .
 *(.ramvectors)
 .ramvectors    0x1fff8000       0xc0 .\CortexM3\ARM_GCC_541\Debug\Cm3Start.o
                0x1fff8000                CyRamVectors

.noinit         0x1fff80c0        0x1
 *(.noinit)
 .noinit        0x1fff80c0        0x1 .\CortexM3\ARM_GCC_541\Debug\Serrure.a(CyLib.o)
                0x1fff80c0                CyResetStatus

.data           0x1fff80c8       0x78 load address 0x000008f0
                0x1fff80c8                __cy_region_start_data = .
 *(.jcr)
 .jcr           0x1fff80c8        0x0 c:/program files (x86)/cypress/psoc creator/4.2/psoc creator/import/gnu/arm/5.4.1/bin/../lib/gcc/arm-none-eabi/5.4.1/armv7-m/crtbegin.o
 .jcr           0x1fff80c8        0x4 c:/program files (x86)/cypress/psoc creator/4.2/psoc creator/import/gnu/arm/5.4.1/bin/../lib/gcc/arm-none-eabi/5.4.1/armv7-m/crtend.o
 *(.got.plt)
 *(.got)
 *(.shdata)
 *(.data .data.* .gnu.linkonce.d.*)
 .data          0x1fff80cc       0x10 .\CortexM3\ARM_GCC_541\Debug\Serrure.a(CyLib.o)
                0x1fff80cc                cydelay_32k_ms
                0x1fff80d0                cydelay_freq_khz
                0x1fff80d4                cydelay_freq_mhz
                0x1fff80d8                cydelay_freq_hz
 .data.impure_data
                0x1fff80dc       0x60 c:/program files (x86)/cypress/psoc creator/4.2/psoc creator/import/gnu/arm/5.4.1/bin/../lib/gcc/arm-none-eabi/5.4.1/../../../../arm-none-eabi/lib/armv7-m\libg_nano.a(lib_a-impure.o)
 .data._impure_ptr
                0x1fff813c        0x4 c:/program files (x86)/cypress/psoc creator/4.2/psoc creator/import/gnu/arm/5.4.1/bin/../lib/gcc/arm-none-eabi/5.4.1/../../../../arm-none-eabi/lib/armv7-m\libg_nano.a(lib_a-impure.o)
                0x1fff813c                _impure_ptr
                0x1fff8140                . = ALIGN (0x8)
 *(.ram)
                0x1fff8140                _edata = .

.igot.plt       0x1fff8140        0x0 load address 0x00000968
 .igot.plt      0x1fff8140        0x0 c:/program files (x86)/cypress/psoc creator/4.2/psoc creator/import/gnu/arm/5.4.1/bin/../lib/gcc/arm-none-eabi/5.4.1/armv7-m/crtbegin.o

.bss            0x1fff8140       0x30 load address 0x00000968
                0x1fff8140                PROVIDE (__bss_start__, .)
 *(.shbss)
 *(.bss .bss.* .gnu.linkonce.b.*)
 .bss           0x1fff8140       0x1c c:/program files (x86)/cypress/psoc creator/4.2/psoc creator/import/gnu/arm/5.4.1/bin/../lib/gcc/arm-none-eabi/5.4.1/armv7-m/crtbegin.o
 .bss           0x1fff815c        0x7 .\CortexM3\ARM_GCC_541\Debug\Serrure.a(UART.o)
                0x1fff815c                UART_errorStatus
                0x1fff815d                UART_initVar
                0x1fff815e                UART_rxBufferRead
                0x1fff815f                UART_rxBufferWrite
                0x1fff8160                UART_rxBufferLoopDetect
                0x1fff8161                UART_rxBufferOverflow
 *(COMMON)
 *fill*         0x1fff8163        0x1 
 COMMON         0x1fff8164        0x5 .\CortexM3\ARM_GCC_541\Debug\Serrure.a(UART.o)
                0x1fff8164                UART_rxBuffer
                0x1fff8170                . = ALIGN (0x8)
 *fill*         0x1fff8169        0x7 
 *(.ram.b)
                0x1fff8170                _end = .
                0x1fff8170                __end = .
                0x1fff8170                PROVIDE (end, .)
                0x1fff8170                PROVIDE (__bss_end__, .)
                0x000008f0                __cy_region_init_ram = LOADADDR (.data)
                0x00000078                __cy_region_init_size_ram = (_edata - ADDR (.data))
                0x00000030                __cy_region_zero_size_ram = (_end - _edata)

.heap           0x1fff8170       0x80 load address 0x00000968
                0x1fff8170                . = _end
                0x1fff81f0                . = (. + 0x80)
 *fill*         0x1fff8170       0x80 
                0x1fff81f0                __cy_heap_limit = .

.stack          0x20007800      0x800
                0x20007800                __cy_stack_limit = .
                0x20008000                . = (. + 0x800)
 *fill*         0x20007800      0x800 
                0x00000001                ASSERT ((__cy_stack_limit >= __cy_heap_limit), region RAM overflowed with stack)
                0x00000000                cy_checksum_exclude_size = (CY_APPL_LOADABLE == 0x1)?SIZEOF (.cy_checksum_exclude):0x0
                0x00000001                ASSERT ((cy_checksum_exclude_size <= CY_CHECKSUM_EXCLUDE_SIZE), CY_BOOT: Section .cy_checksum_exclude size exceedes specified limit.)

.cyloadermeta
 *(.cyloadermeta)

.cyloadablemeta
 *(.cyloadablemeta)

.cyconfigecc    0x80000000      0x6e4
 *(.cyconfigecc)
 .cyconfigecc   0x80000000      0x6e4 .\CortexM3\ARM_GCC_541\Debug\cymetadata.o
                0x80000000                cy_meta_configecc

.cycustnvl      0x90000000        0x4
 *(.cycustnvl)
 .cycustnvl     0x90000000        0x4 .\CortexM3\ARM_GCC_541\Debug\cymetadata.o
                0x90000000                cy_meta_custnvl

.cywolatch      0x90100000        0x4
 *(.cywolatch)
 .cywolatch     0x90100000        0x4 .\CortexM3\ARM_GCC_541\Debug\cymetadata.o
                0x90100000                cy_meta_wonvl

.cyeeprom       0x90200000        0x0
 *(.cyeeprom)
                0x00000001                ASSERT ((. <= ((0x90200000 + ee_offset) + ee_size)), .cyeeprom data will not fit in EEPROM)

.cyflashprotect
                0x90400000      0x100
 *(.cyflashprotect)
 .cyflashprotect
                0x90400000      0x100 .\CortexM3\ARM_GCC_541\Debug\cymetadata.o
                0x90400000                cy_meta_flashprotect

.cymeta         0x90500000        0xc
 *(.cymeta)
 .cymeta        0x90500000        0xc .\CortexM3\ARM_GCC_541\Debug\cymetadata.o
                0x90500000                cy_metadata

.rel.dyn        0x00000968        0x0 load address 0x9050000c
 .rel.iplt      0x00000968        0x0 c:/program files (x86)/cypress/psoc creator/4.2/psoc creator/import/gnu/arm/5.4.1/bin/../lib/gcc/arm-none-eabi/5.4.1/armv7-m/crtbegin.o

.stab
 *(.stab)

.stabstr
 *(.stabstr)

.debug
 *(.debug)

.line
 *(.line)

.debug_srcinfo
 *(.debug_srcinfo)

.debug_sfnames
 *(.debug_sfnames)

.debug_aranges  0x00000000      0x770
 *(.debug_aranges)
 .debug_aranges
                0x00000000       0x20 .\CortexM3\ARM_GCC_541\Debug\main.o
 .debug_aranges
                0x00000020       0x58 .\CortexM3\ARM_GCC_541\Debug\cyfitter_cfg.o
 .debug_aranges
                0x00000078       0x18 .\CortexM3\ARM_GCC_541\Debug\cymetadata.o
 .debug_aranges
                0x00000090       0x48 .\CortexM3\ARM_GCC_541\Debug\Cm3Start.o
 .debug_aranges
                0x000000d8      0x2a0 .\CortexM3\ARM_GCC_541\Debug\Serrure.a(CyLib.o)
 .debug_aranges
                0x00000378       0x98 .\CortexM3\ARM_GCC_541\Debug\Serrure.a(cyPm.o)
 .debug_aranges
                0x00000410       0xf0 .\CortexM3\ARM_GCC_541\Debug\Serrure.a(UART.o)
 .debug_aranges
                0x00000500       0x20 .\CortexM3\ARM_GCC_541\Debug\Serrure.a(UART_INT.o)
 .debug_aranges
                0x00000520       0x70 .\CortexM3\ARM_GCC_541\Debug\Serrure.a(UART_IntClock.o)
 .debug_aranges
                0x00000590       0x80 .\CortexM3\ARM_GCC_541\Debug\Serrure.a(rfid.o)
 .debug_aranges
                0x00000610       0x38 .\CortexM3\ARM_GCC_541\Debug\Serrure.a(led.o)
 .debug_aranges
                0x00000648       0x20 .\CortexM3\ARM_GCC_541\Debug\Serrure.a(CyBootAsmGnu.o)
 .debug_aranges
                0x00000668       0x88 .\CortexM3\ARM_GCC_541\Debug\Serrure.a(CyFlash.o)
 .debug_aranges
                0x000006f0       0x80 .\CortexM3\ARM_GCC_541\Debug\Serrure.a(CySpc.o)

.debug_pubnames
 *(.debug_pubnames)

.debug_info     0x00000000     0x4667
 *(.debug_info .gnu.linkonce.wi.*)
 .debug_info    0x00000000      0x116 .\CortexM3\ARM_GCC_541\Debug\main.o
 .debug_info    0x00000116      0x595 .\CortexM3\ARM_GCC_541\Debug\cyfitter_cfg.o
 .debug_info    0x000006ab      0x139 .\CortexM3\ARM_GCC_541\Debug\cymetadata.o
 .debug_info    0x000007e4      0x3bb .\CortexM3\ARM_GCC_541\Debug\Cm3Start.o
 .debug_info    0x00000b9f     0x1374 .\CortexM3\ARM_GCC_541\Debug\Serrure.a(CyLib.o)
 .debug_info    0x00001f13      0xa2a .\CortexM3\ARM_GCC_541\Debug\Serrure.a(cyPm.o)
 .debug_info    0x0000293d      0x72d .\CortexM3\ARM_GCC_541\Debug\Serrure.a(UART.o)
 .debug_info    0x0000306a      0x14c .\CortexM3\ARM_GCC_541\Debug\Serrure.a(UART_INT.o)
 .debug_info    0x000031b6      0x283 .\CortexM3\ARM_GCC_541\Debug\Serrure.a(UART_IntClock.o)
 .debug_info    0x00003439      0x4cf .\CortexM3\ARM_GCC_541\Debug\Serrure.a(rfid.o)
 .debug_info    0x00003908      0x11f .\CortexM3\ARM_GCC_541\Debug\Serrure.a(led.o)
 .debug_info    0x00003a27       0xa3 .\CortexM3\ARM_GCC_541\Debug\Serrure.a(CyBootAsmGnu.o)
 .debug_info    0x00003aca      0x64d .\CortexM3\ARM_GCC_541\Debug\Serrure.a(CyFlash.o)
 .debug_info    0x00004117      0x550 .\CortexM3\ARM_GCC_541\Debug\Serrure.a(CySpc.o)

.debug_abbrev   0x00000000     0x1215
 *(.debug_abbrev)
 .debug_abbrev  0x00000000       0xa1 .\CortexM3\ARM_GCC_541\Debug\main.o
 .debug_abbrev  0x000000a1      0x20d .\CortexM3\ARM_GCC_541\Debug\cyfitter_cfg.o
 .debug_abbrev  0x000002ae       0x77 .\CortexM3\ARM_GCC_541\Debug\cymetadata.o
 .debug_abbrev  0x00000325      0x1e8 .\CortexM3\ARM_GCC_541\Debug\Cm3Start.o
 .debug_abbrev  0x0000050d      0x254 .\CortexM3\ARM_GCC_541\Debug\Serrure.a(CyLib.o)
 .debug_abbrev  0x00000761      0x1ab .\CortexM3\ARM_GCC_541\Debug\Serrure.a(cyPm.o)
 .debug_abbrev  0x0000090c      0x16f .\CortexM3\ARM_GCC_541\Debug\Serrure.a(UART.o)
 .debug_abbrev  0x00000a7b       0x8a .\CortexM3\ARM_GCC_541\Debug\Serrure.a(UART_INT.o)
 .debug_abbrev  0x00000b05      0x139 .\CortexM3\ARM_GCC_541\Debug\Serrure.a(UART_IntClock.o)
 .debug_abbrev  0x00000c3e      0x1f8 .\CortexM3\ARM_GCC_541\Debug\Serrure.a(rfid.o)
 .debug_abbrev  0x00000e36       0x90 .\CortexM3\ARM_GCC_541\Debug\Serrure.a(led.o)
 .debug_abbrev  0x00000ec6       0x14 .\CortexM3\ARM_GCC_541\Debug\Serrure.a(CyBootAsmGnu.o)
 .debug_abbrev  0x00000eda      0x1a7 .\CortexM3\ARM_GCC_541\Debug\Serrure.a(CyFlash.o)
 .debug_abbrev  0x00001081      0x194 .\CortexM3\ARM_GCC_541\Debug\Serrure.a(CySpc.o)

.debug_line     0x00000000     0x1e92
 *(.debug_line)
 .debug_line    0x00000000      0x170 .\CortexM3\ARM_GCC_541\Debug\main.o
 .debug_line    0x00000170      0x1f5 .\CortexM3\ARM_GCC_541\Debug\cyfitter_cfg.o
 .debug_line    0x00000365      0x141 .\CortexM3\ARM_GCC_541\Debug\cymetadata.o
 .debug_line    0x000004a6      0x234 .\CortexM3\ARM_GCC_541\Debug\Cm3Start.o
 .debug_line    0x000006da      0x816 .\CortexM3\ARM_GCC_541\Debug\Serrure.a(CyLib.o)
 .debug_line    0x00000ef0      0x367 .\CortexM3\ARM_GCC_541\Debug\Serrure.a(cyPm.o)
 .debug_line    0x00001257      0x302 .\CortexM3\ARM_GCC_541\Debug\Serrure.a(UART.o)
 .debug_line    0x00001559       0x81 .\CortexM3\ARM_GCC_541\Debug\Serrure.a(UART_INT.o)
 .debug_line    0x000015da      0x17c .\CortexM3\ARM_GCC_541\Debug\Serrure.a(UART_IntClock.o)
 .debug_line    0x00001756      0x1cc .\CortexM3\ARM_GCC_541\Debug\Serrure.a(rfid.o)
 .debug_line    0x00001922       0x90 .\CortexM3\ARM_GCC_541\Debug\Serrure.a(led.o)
 .debug_line    0x000019b2       0x66 .\CortexM3\ARM_GCC_541\Debug\Serrure.a(CyBootAsmGnu.o)
 .debug_line    0x00001a18      0x21a .\CortexM3\ARM_GCC_541\Debug\Serrure.a(CyFlash.o)
 .debug_line    0x00001c32      0x260 .\CortexM3\ARM_GCC_541\Debug\Serrure.a(CySpc.o)

.debug_frame    0x00000000     0x1388
 *(.debug_frame)
 .debug_frame   0x00000000       0x2c .\CortexM3\ARM_GCC_541\Debug\main.o
 .debug_frame   0x0000002c       0xe4 .\CortexM3\ARM_GCC_541\Debug\cyfitter_cfg.o
 .debug_frame   0x00000110       0xb8 .\CortexM3\ARM_GCC_541\Debug\Cm3Start.o
 .debug_frame   0x000001c8      0x738 .\CortexM3\ARM_GCC_541\Debug\Serrure.a(CyLib.o)
 .debug_frame   0x00000900      0x1f8 .\CortexM3\ARM_GCC_541\Debug\Serrure.a(cyPm.o)
 .debug_frame   0x00000af8      0x25c .\CortexM3\ARM_GCC_541\Debug\Serrure.a(UART.o)
 .debug_frame   0x00000d54       0x20 .\CortexM3\ARM_GCC_541\Debug\Serrure.a(UART_INT.o)
 .debug_frame   0x00000d74       0xe0 .\CortexM3\ARM_GCC_541\Debug\Serrure.a(UART_IntClock.o)
 .debug_frame   0x00000e54      0x114 .\CortexM3\ARM_GCC_541\Debug\Serrure.a(rfid.o)
 .debug_frame   0x00000f68       0x50 .\CortexM3\ARM_GCC_541\Debug\Serrure.a(led.o)
 .debug_frame   0x00000fb8      0x194 .\CortexM3\ARM_GCC_541\Debug\Serrure.a(CyFlash.o)
 .debug_frame   0x0000114c      0x180 .\CortexM3\ARM_GCC_541\Debug\Serrure.a(CySpc.o)
 .debug_frame   0x000012cc       0x20 c:/program files (x86)/cypress/psoc creator/4.2/psoc creator/import/gnu/arm/5.4.1/bin/../lib/gcc/arm-none-eabi/5.4.1/../../../../arm-none-eabi/lib/armv7-m\libg_nano.a(lib_a-errno.o)
 .debug_frame   0x000012ec       0x28 c:/program files (x86)/cypress/psoc creator/4.2/psoc creator/import/gnu/arm/5.4.1/bin/../lib/gcc/arm-none-eabi/5.4.1/../../../../arm-none-eabi/lib/armv7-m\libg_nano.a(lib_a-exit.o)
 .debug_frame   0x00001314       0x2c c:/program files (x86)/cypress/psoc creator/4.2/psoc creator/import/gnu/arm/5.4.1/bin/../lib/gcc/arm-none-eabi/5.4.1/../../../../arm-none-eabi/lib/armv7-m\libg_nano.a(lib_a-init.o)
 .debug_frame   0x00001340       0x28 c:/program files (x86)/cypress/psoc creator/4.2/psoc creator/import/gnu/arm/5.4.1/bin/../lib/gcc/arm-none-eabi/5.4.1/../../../../arm-none-eabi/lib/armv7-m\libg_nano.a(lib_a-memcpy-stub.o)
 .debug_frame   0x00001368       0x20 c:/program files (x86)/cypress/psoc creator/4.2/psoc creator/import/gnu/arm/5.4.1/bin/../lib/gcc/arm-none-eabi/5.4.1/../../../../arm-none-eabi/lib/armv7-m\libg_nano.a(lib_a-memset.o)

.debug_str      0x00000000     0x197d
 *(.debug_str)
 .debug_str     0x00000000      0x196 .\CortexM3\ARM_GCC_541\Debug\main.o
                                0x1de (size before relaxing)
 .debug_str     0x00000196      0x1bc .\CortexM3\ARM_GCC_541\Debug\cyfitter_cfg.o
                                0x357 (size before relaxing)
 .debug_str     0x00000352       0x7f .\CortexM3\ARM_GCC_541\Debug\cymetadata.o
                                0x1f7 (size before relaxing)
 .debug_str     0x000003d1      0x144 .\CortexM3\ARM_GCC_541\Debug\Cm3Start.o
                                0x31d (size before relaxing)
 .debug_str     0x00000515      0x854 .\CortexM3\ARM_GCC_541\Debug\Serrure.a(CyLib.o)
                                0xa5a (size before relaxing)
 .debug_str     0x00000d69      0x365 .\CortexM3\ARM_GCC_541\Debug\Serrure.a(cyPm.o)
                                0x746 (size before relaxing)
 .debug_str     0x000010ce      0x32f .\CortexM3\ARM_GCC_541\Debug\Serrure.a(UART.o)
                                0x557 (size before relaxing)
 .debug_str     0x000013fd       0x53 .\CortexM3\ARM_GCC_541\Debug\Serrure.a(UART_INT.o)
                                0x25e (size before relaxing)
 .debug_str     0x00001450      0x183 .\CortexM3\ARM_GCC_541\Debug\Serrure.a(UART_IntClock.o)
                                0x349 (size before relaxing)
 .debug_str     0x000015d3       0xf1 .\CortexM3\ARM_GCC_541\Debug\Serrure.a(rfid.o)
                                0x328 (size before relaxing)
 .debug_str     0x000016c4       0x52 .\CortexM3\ARM_GCC_541\Debug\Serrure.a(led.o)
                                0x1eb (size before relaxing)
 .debug_str     0x00001716      0x1bb .\CortexM3\ARM_GCC_541\Debug\Serrure.a(CyFlash.o)
                                0x3d3 (size before relaxing)
 .debug_str     0x000018d1       0xac .\CortexM3\ARM_GCC_541\Debug\Serrure.a(CySpc.o)
                                0x34b (size before relaxing)

.debug_loc      0x00000000     0x1feb
 *(.debug_loc)
 .debug_loc     0x00000000      0x25a .\CortexM3\ARM_GCC_541\Debug\cyfitter_cfg.o
 .debug_loc     0x0000025a      0x144 .\CortexM3\ARM_GCC_541\Debug\Cm3Start.o
 .debug_loc     0x0000039e      0xa11 .\CortexM3\ARM_GCC_541\Debug\Serrure.a(CyLib.o)
 .debug_loc     0x00000daf      0x1e4 .\CortexM3\ARM_GCC_541\Debug\Serrure.a(cyPm.o)
 .debug_loc     0x00000f93      0x34e .\CortexM3\ARM_GCC_541\Debug\Serrure.a(UART.o)
 .debug_loc     0x000012e1       0x45 .\CortexM3\ARM_GCC_541\Debug\Serrure.a(UART_INT.o)
 .debug_loc     0x00001326      0x12c .\CortexM3\ARM_GCC_541\Debug\Serrure.a(UART_IntClock.o)
 .debug_loc     0x00001452       0xa0 .\CortexM3\ARM_GCC_541\Debug\Serrure.a(rfid.o)
 .debug_loc     0x000014f2       0x42 .\CortexM3\ARM_GCC_541\Debug\Serrure.a(led.o)
 .debug_loc     0x00001534      0x3b2 .\CortexM3\ARM_GCC_541\Debug\Serrure.a(CyFlash.o)
 .debug_loc     0x000018e6      0x705 .\CortexM3\ARM_GCC_541\Debug\Serrure.a(CySpc.o)

.debug_macinfo
 *(.debug_macinfo)

.debug_ranges   0x00000000      0x6a8
 *(.debug_ranges)
 .debug_ranges  0x00000000       0x10 .\CortexM3\ARM_GCC_541\Debug\main.o
 .debug_ranges  0x00000010       0x48 .\CortexM3\ARM_GCC_541\Debug\cyfitter_cfg.o
 .debug_ranges  0x00000058       0x38 .\CortexM3\ARM_GCC_541\Debug\Cm3Start.o
 .debug_ranges  0x00000090      0x290 .\CortexM3\ARM_GCC_541\Debug\Serrure.a(CyLib.o)
 .debug_ranges  0x00000320       0x88 .\CortexM3\ARM_GCC_541\Debug\Serrure.a(cyPm.o)
 .debug_ranges  0x000003a8       0xe0 .\CortexM3\ARM_GCC_541\Debug\Serrure.a(UART.o)
 .debug_ranges  0x00000488       0x10 .\CortexM3\ARM_GCC_541\Debug\Serrure.a(UART_INT.o)
 .debug_ranges  0x00000498       0x60 .\CortexM3\ARM_GCC_541\Debug\Serrure.a(UART_IntClock.o)
 .debug_ranges  0x000004f8       0xa0 .\CortexM3\ARM_GCC_541\Debug\Serrure.a(rfid.o)
 .debug_ranges  0x00000598       0x28 .\CortexM3\ARM_GCC_541\Debug\Serrure.a(led.o)
 .debug_ranges  0x000005c0       0x78 .\CortexM3\ARM_GCC_541\Debug\Serrure.a(CyFlash.o)
 .debug_ranges  0x00000638       0x70 .\CortexM3\ARM_GCC_541\Debug\Serrure.a(CySpc.o)

.comment        0x00000000       0x6e
 .comment       0x00000000       0x6e .\CortexM3\ARM_GCC_541\Debug\main.o
                                 0x6f (size before relaxing)
 .comment       0x0000006e       0x6f .\CortexM3\ARM_GCC_541\Debug\cyfitter_cfg.o
 .comment       0x0000006e       0x6f .\CortexM3\ARM_GCC_541\Debug\cymetadata.o
 .comment       0x0000006e       0x6f .\CortexM3\ARM_GCC_541\Debug\Cm3Start.o
 .comment       0x0000006e       0x6f .\CortexM3\ARM_GCC_541\Debug\Serrure.a(CyLib.o)
 .comment       0x0000006e       0x6f .\CortexM3\ARM_GCC_541\Debug\Serrure.a(cyPm.o)
 .comment       0x0000006e       0x6f .\CortexM3\ARM_GCC_541\Debug\Serrure.a(UART.o)
 .comment       0x0000006e       0x6f .\CortexM3\ARM_GCC_541\Debug\Serrure.a(UART_INT.o)
 .comment       0x0000006e       0x6f .\CortexM3\ARM_GCC_541\Debug\Serrure.a(UART_IntClock.o)
 .comment       0x0000006e       0x6f .\CortexM3\ARM_GCC_541\Debug\Serrure.a(rfid.o)
 .comment       0x0000006e       0x6f .\CortexM3\ARM_GCC_541\Debug\Serrure.a(led.o)
 .comment       0x0000006e       0x6f .\CortexM3\ARM_GCC_541\Debug\Serrure.a(CyFlash.o)
 .comment       0x0000006e       0x6f .\CortexM3\ARM_GCC_541\Debug\Serrure.a(CySpc.o)

.debug_weaknames
 *(.debug_weaknames)

.debug_funcnames
 *(.debug_funcnames)

.debug_typenames
 *(.debug_typenames)

.debug_varnames
 *(.debug_varnames)

.note.gnu.arm.ident
 *(.note.gnu.arm.ident)

.ARM.attributes
                0x00000000       0x29
 *(.ARM.attributes)
 .ARM.attributes
                0x00000000       0x1d c:/program files (x86)/cypress/psoc creator/4.2/psoc creator/import/gnu/arm/5.4.1/bin/../lib/gcc/arm-none-eabi/5.4.1/armv7-m/crti.o
 .ARM.attributes
                0x0000001d       0x2d c:/program files (x86)/cypress/psoc creator/4.2/psoc creator/import/gnu/arm/5.4.1/bin/../lib/gcc/arm-none-eabi/5.4.1/armv7-m/crtbegin.o
 .ARM.attributes
                0x0000004a       0x1b c:/program files (x86)/cypress/psoc creator/4.2/psoc creator/import/gnu/arm/5.4.1/bin/../lib/gcc/arm-none-eabi/5.4.1/../../../../arm-none-eabi/lib/armv7-m/crt0.o
 .ARM.attributes
                0x00000065       0x33 .\CortexM3\ARM_GCC_541\Debug\main.o
 .ARM.attributes
                0x00000098       0x33 .\CortexM3\ARM_GCC_541\Debug\cyfitter_cfg.o
 .ARM.attributes
                0x000000cb       0x33 .\CortexM3\ARM_GCC_541\Debug\cymetadata.o
 .ARM.attributes
                0x000000fe       0x33 .\CortexM3\ARM_GCC_541\Debug\Cm3Start.o
 .ARM.attributes
                0x00000131       0x33 .\CortexM3\ARM_GCC_541\Debug\Serrure.a(CyLib.o)
 .ARM.attributes
                0x00000164       0x33 .\CortexM3\ARM_GCC_541\Debug\Serrure.a(cyPm.o)
 .ARM.attributes
                0x00000197       0x33 .\CortexM3\ARM_GCC_541\Debug\Serrure.a(UART.o)
 .ARM.attributes
                0x000001ca       0x33 .\CortexM3\ARM_GCC_541\Debug\Serrure.a(UART_INT.o)
 .ARM.attributes
                0x000001fd       0x33 .\CortexM3\ARM_GCC_541\Debug\Serrure.a(UART_IntClock.o)
 .ARM.attributes
                0x00000230       0x33 .\CortexM3\ARM_GCC_541\Debug\Serrure.a(rfid.o)
 .ARM.attributes
                0x00000263       0x33 .\CortexM3\ARM_GCC_541\Debug\Serrure.a(led.o)
 .ARM.attributes
                0x00000296       0x21 .\CortexM3\ARM_GCC_541\Debug\Serrure.a(CyBootAsmGnu.o)
 .ARM.attributes
                0x000002b7       0x33 .\CortexM3\ARM_GCC_541\Debug\Serrure.a(CyFlash.o)
 .ARM.attributes
                0x000002ea       0x33 .\CortexM3\ARM_GCC_541\Debug\Serrure.a(CySpc.o)
 .ARM.attributes
                0x0000031d       0x2d c:/program files (x86)/cypress/psoc creator/4.2/psoc creator/import/gnu/arm/5.4.1/bin/../lib/gcc/arm-none-eabi/5.4.1/../../../../arm-none-eabi/lib/armv7-m\libg_nano.a(lib_a-errno.o)
 .ARM.attributes
                0x0000034a       0x2d c:/program files (x86)/cypress/psoc creator/4.2/psoc creator/import/gnu/arm/5.4.1/bin/../lib/gcc/arm-none-eabi/5.4.1/../../../../arm-none-eabi/lib/armv7-m\libg_nano.a(lib_a-exit.o)
 .ARM.attributes
                0x00000377       0x2d c:/program files (x86)/cypress/psoc creator/4.2/psoc creator/import/gnu/arm/5.4.1/bin/../lib/gcc/arm-none-eabi/5.4.1/../../../../arm-none-eabi/lib/armv7-m\libg_nano.a(lib_a-impure.o)
 .ARM.attributes
                0x000003a4       0x2d c:/program files (x86)/cypress/psoc creator/4.2/psoc creator/import/gnu/arm/5.4.1/bin/../lib/gcc/arm-none-eabi/5.4.1/../../../../arm-none-eabi/lib/armv7-m\libg_nano.a(lib_a-init.o)
 .ARM.attributes
                0x000003d1       0x2d c:/program files (x86)/cypress/psoc creator/4.2/psoc creator/import/gnu/arm/5.4.1/bin/../lib/gcc/arm-none-eabi/5.4.1/../../../../arm-none-eabi/lib/armv7-m\libg_nano.a(lib_a-memcpy-stub.o)
 .ARM.attributes
                0x000003fe       0x2d c:/program files (x86)/cypress/psoc creator/4.2/psoc creator/import/gnu/arm/5.4.1/bin/../lib/gcc/arm-none-eabi/5.4.1/../../../../arm-none-eabi/lib/armv7-m\libg_nano.a(lib_a-memset.o)
 .ARM.attributes
                0x0000042b       0x2d c:/program files (x86)/cypress/psoc creator/4.2/psoc creator/import/gnu/arm/5.4.1/bin/../lib/gcc/arm-none-eabi/5.4.1/armv7-m/crtend.o
 .ARM.attributes
                0x00000458       0x1d c:/program files (x86)/cypress/psoc creator/4.2/psoc creator/import/gnu/arm/5.4.1/bin/../lib/gcc/arm-none-eabi/5.4.1/armv7-m/crtn.o

/DISCARD/
 *(.note.GNU-stack)
OUTPUT(P:\Travaux pratique\Electronique\Mini projet Serrure\Emilio Work Space\Serrure.cydsn\CortexM3\ARM_GCC_541\Debug\Serrure.elf elf32-littlearm)
